:100000000C94FA020C9419030C9419030C94190320
:100010000C9419030C9419030C9419030C941903F0
:100020000C9419030C9419030C945D230C94332441
:100030000C94311E0C9419030C9419030C9419039D
:100040000C9419030C9419030C9419030C941903C0
:100050000C9419030C94B91E0C9419030C941903F5
:100060000C9419030C9419030C9419030C941903A0
:100070000C9419030C9419030C9419030C94190390
:100080000C9419030C9419030C9419030C94190380
:100090000C9419030C941903E005E0050C060C06FA
:1000A00074069206AA07AA079D0636074707470760
:1000B000A424CB24C325CB24C32517253A25C32547
:1000C0009125A025000000000000000080808080B5
:1000D0000000000000000000000000000000000020
:1000E0000000000000C0C080000000000000000010
:1000F0000000000000000000000000000000000000
:1001000000000000000000000000000000000000EF
:1001100000008080808080800000000000000000DF
:1001200000000000000000000000000000000000CF
:10013000000000000000808080000000000000003F
:100140000000000000000000000000F0FF0F03FFAF
:10015000FC80000000F8F86030F8F02030F8F00083
:100160000000383838F9F901000000000000E0F024
:10017000381818F8F89818000000E0F0F0383878CF
:10018000F0E000000000000000000000000000009F
:100190000000FFFF03030303FFFF78000000F8F8EF
:1001A00000000000F8F800000000F8F8F0203078B7
:1001B000F8F000000000FFFFFF00C0F0F838080072
:1001C000000000000000000000C0FE7F0F0E0E0EB9
:1001D0007FFFF00000FFFF0000FFFF0000FFFF00B7
:1001E0000000E0E0E0FFFFE0E0E000000000BCFD18
:1001F000E7E6E6E3E3C1800000003F7F78E0E0F05F
:100200007F3F000000000000000000000000000030
:100210000000FFFF070707070303000000007FFF40
:10022000F0602030FFFF00000000FFFF0000000032
:10023000FFFF00000000FFFFFF071F7FF8E08000C6
:1002400000000000000000000000000000000000AE
:10025000000000000000000000000000000000009E
:100260000000000000000000000000000003070F75
:100270000C0C0C0C0C070300000000000000000038
:10028000000000000000000000000000000000006E
:10029000000000000000000000000000000000005E
:1002A000000000000000000000000000000000004E
:1002B000000000000000000000000000000000003E
:1002C0000000000029003A003B003C003D003E00D9
:1002D0003F00400041004200430044004500490007
:1002E0004C000000A80035001E001F002000210067
:1002F0002200230024002500260027002D002E00C8
:1003000000002A004B0000002B00000014001A001F
:100310000800150017001C0018000C001200130044
:100320002F00300031004E000000E000000004000B
:100330001600070009000A000B000D000E000F0058
:100340003300340028000000000000000000E1003D
:100350001D001B00060019000500110010003600EA
:10036000370038000000E1000000520000000000EB
:10037000E3000000E2000000000000002C0000008C
:1003800000000000000000000151500051004F002B
:100390000100010001000100010001000100010055
:1003A0000100005C010001000100460001000000A6
:1003B0000100010001000100010001000100010035
:1003C0000100010001000100010001000000010026
:1003D0004A000000010000000100010001000100CE
:1003E0000100010001000100010001000100010005
:1003F00001004D0000003900000001000100010073
:1004000001000100010001000100010001000100E4
:10041000AE0000000000000000000100010001002B
:1004200001000100010001000100010001000100C4
:100430000000A8000000A90000000000010000006A
:1004400001000000000000000100000000000000AA
:10045000010000000100AC00AA00AB0000AE00AF3C
:1004600000DA0281FFD9F1DB20A4A62EAF00A0C0E4
:1004700000A1C800AED580A81FD300408D14200075
:10048000140361006D00690067006F007000750063
:100490006E006B00000014036800610065007300CB
:1004A000620061006500720074000000040309042A
:1004B00009023B00020100A0FA0904000001030147
:1004C00001000921110100012240000705810308F4
:1004D00000010904010001030000000921110100CD
:1004E0000122B6000705820320000112010002006C
:1004F000000008EDFE0518010001020001050109D8
:1005000002A10185020901A10005091901290815A7
:100510000025019508750181020501093009311591
:1005200081257F95027508810609381581257F95FB
:100530000175088106050C0A38021581257F950191
:1005400075088106C0C005010980A1018503190154
:100550002AB700150126B700950175108100C00566
:100560000C0901A101850419012AA002150126A088
:1005700002950175108100C005010906A1018506DB
:10058000050719E029E71500250195087501810285
:100590000507190029EF1500250195F07501810265
:1005A0000508190129059505750191029501750345
:1005B0009101C005010906A101050719E029E71508
:1005C00000250195087501810295017508810105D5
:1005D00007190029FF150026FF0095067508810000
:1005E0000508190129059505750191029501750305
:1005F0009101C00011241FBECFEFD0E2DEBFCDBFFE
:1006000011E0A0E0B1E0E2EFFCE400E00BBF02C0CB
:1006100007900D92A23BB107D9F725E0A2EBB1E01C
:1006200001C01D92A435B207E1F70E9425140C9475
:1006300077260C940000811109C0611102C08AEA7A
:1006400001C089EA0E948E0581E0089580E0089546
:1006500060E072E084EC90E00E945D1780E0089515
:1006600081E0089581E008950C94320308950C947C
:1006700036031F93CF93DF9300D000D01F92CDB7E6
:10068000DEB749835A836B833091B50189819A81A2
:10069000311114C0662359F0222349F00E94E70962
:1006A000182F682F89819A810E94900903C00E94A7
:1006B000BB09182F69817A81812F04C00E94E70944
:1006C00069817A810F900F900F900F900F90DF91BA
:1006D000CF911F910C946F11FC01262F4081518105
:1006E0006281738184810C94390381E00895CF93F2
:1006F000DF93EC0160E00E946C03BE01DF91CF91BB
:100700000C9437030C94B8120C94B41208950E9400
:100710003A080E9486032FEF84E39CE0215080403A
:100720009040E1F700C000000C94DF1E0F931F9370
:10073000CF93DF938C0161E00E946C03EC01B80160
:100740000E9434038823F1F1B801CE010E946B1B93
:100750008823C1F1B801CE010E941819882391F1B4
:10076000B801CE010E94C71A882361F1F801828185
:10077000882309F1CB358DE5D807C1F050F4C115B8
:10078000FCE5DF0781F0CF3DDC45A9F40E941E0F98
:1007900019C0CC35EDE5DE0761F0CD35DD4559F406
:1007A0000E94610E08C00E9487030CC00E946A0E5E
:1007B00002C00E946D0EC801DF91CF911F910F9171
:1007C0000C94300380E0DF91CF911F910F91089539
:1007D0000E94111E0E9403040C94CE180E9406046D
:1007E0000C94171E08950C94F20381E008950C9464
:1007F000F5030895CF93C82F0E94F3038C2F0E9416
:10080000F703CF91089580E00C94FA030E94D61C60
:100810000C94FA030E94D61C9091B401891721F020
:100820008093B4010C94FA030895CF93DF93CDB76E
:10083000DEB72B970FB6F894DEBF0FBECDBF4F8348
:10084000588769877A878B8761110E94AD0D9E0159
:100850002F5F3F4F86E0F90111928A95E9F785E015
:10086000FE013796D90101900D928A95E1F78981B1
:100870009A814C815D81452B31F09F3F31F491E0AD
:100880008F3F19F403C091E001C090E090FF09C0D0
:1008900049815A816B817C818D819E810E94CE0C21
:1008A00005C0C9010E9475038111F2CF2B960FB6C6
:1008B000F894DEBF0FBECDBFDF91CF910895FC014C
:1008C000808191810E94290A0895CF93882309F499
:1008D000A4C0C82F8238C1F40E94D61C81FD9DC0DF
:1008E00069E380910201909103010E94CC1D0E9456
:1008F000CF0D2FEF81EE94E0215080409040E1F742
:1009000000C0000069E319C0833801F50E94D61CBD
:1009100080FD83C063E580910201909103010E94F4
:10092000CC1D0E94CF0D2FEF81EE94E0215080402E
:100930009040E1F700C0000063E5809102019091D2
:1009400003010E94D71DCF910C94CF0D8438C1F4C0
:100950000E94D61C82FD61C067E4809102019091E3
:1009600003010E94CC1D0E94CF0D2FEF81EE94E079
:10097000215080409040E1F700C0000067E4DDCFE7
:100980008CEF8C0F813AD0F46C2F80910201909102
:1009900003010E944C1D882349F06C2F80910201B5
:1009A000909103010E94D71D0E94CF0D6C2F809162
:1009B0000201909103010E94CC1DC5CF80E28C0FF3
:1009C000883048F4C77081E001C0880FCA95EAF703
:1009D0000E94900DB8CFEBE5EC0FE33040F4F0E06F
:1009E000E25BFE4F808190E0CF910C940A1DE8E518
:1009F000EC0FE73150F4F0E0EE0FFF1FE05EFE4F2A
:100A000080819181CF910C94201DCD3E30F08C2FB0
:100A10000E94AA14CF910C947C15CF91089588233D
:100A200009F464C0823879F40E94D61C81FF5EC04C
:100A300069E380910201909103010E94CC1D0E9404
:100A4000CF0D69E310C08338B1F40E94D61C80FF3B
:100A50004DC063E580910201909103010E94CC1D7D
:100A60000E94CF0D63E580910201909103010E94E5
:100A7000D71D0C94CF0D843879F40E94D61C82FFC8
:100A800035C067E480910201909103010E94CC1D62
:100A90000E94CF0D67E4E7CF9CEF980F913A10F4D6
:100AA000682FE1CF90E2980F983050F4877091E072
:100AB00001C0990F8A95EAF7892F0E94960DD9CF28
:100AC0009BE5980F933020F480E090E00C940A1D91
:100AD00098E5980F973120F480E090E00C94201D69
:100AE0008D3E20F00E9405150C947C1508951F93EF
:100AF000CF93DF93182FEB010E946504209741F0FC
:100B00008FE99FE00197F1F700C000002197F6CF31
:100B1000812FDF91CF911F910C940F05893319F02C
:100B200060E070E002C060E570E00C947705882317
:100B300021F00E94900D0C94CF0D0895882321F090
:100B40000E94960D0C94CF0D0895CF92DF92EF92F4
:100B5000FF920F931F93CF93DF937C01D62FC72F64
:100B6000FC011281058102950F700E94860D882379
:100B7000B9F01123A9F08C2F807F803421F080E21E
:100B80008D0F883068F080910C0382FD09C082E0EF
:100B90000E942F0E0E94860D91E0D82ED92601C00A
:100BA000D12CCC2EC2948FE0C8228C2D90E08C30BA
:100BB000910508F0CFC1FC01E45BFF4F0C941F26A8
:100BC0008C2F807FCF70882311F0C295C07F1123B6
:100BD00099F0CC2309F4AAC180E28D0F883010F07F
:100BE000D11104C08C2F0E94900D03C08C2F0E9445
:100BF000A00D0E94CF0D9AC18D2F0E940F05CC230E
:100C000009F4A8C180E28D0F883038F1DD2329F185
:100C10008C2F0E94A60D24C08C2F807FCF70803235
:100C200011F0C295C07FDD2319F0D130A1F13DC094
:100C300080910C0382FF17C0112349F0CC2329F0C7
:100C40008C2F0E94900D0E94CF0D80E070C180E03B
:100C50000E940F05CC2309F47DC18C2F0E94960DB4
:100C60000E94CF0D77C1112371F0002341F00130B4
:100C700031F40E94B00D8C2B0E94B80D6BC10E9404
:100C8000B00D8C2B1DC0002319F0013009F462C196
:100C90000E94C50D25C0112321F0063008F05AC16D
:100CA0000EC0053008F056C11BC0112361F00023AF
:100CB00031F0F701858180FF39C18F7085838C2FDA
:100CC0000E94970547C1002359F0D93309F03FC16D
:100CD000FFEF07EE13E0F15000401040E1F735C19F
:100CE0008C2F0E949E0536C18C2F86958695837029
:100CF00019F0813061F02EC1112321F08D2F9C2F2E
:100D0000937002C080E090E00E940A1D2BC1112365
:100D100021F08D2F9C2F937002C080E090E00E9404
:100D2000201D20C18D2F112319F00E94AA1402C08A
:100D30000E9405150E947C1515C18C2F837009F047
:100D400047C011110BC12D2F229526952770220F18
:100D5000220F6D2F6F70862F90E0A0E0B0E0022E82
:100D600004C0880F991FAA1FBB1F0A94D2F7D4FF93
:100D700010C04FE050E060E070E004C0440F551F29
:100D8000661F771F2A95D2F740955095609570950C
:100D900003C040E050E0BA01C695C695C3708A0111
:100DA0009B01082B192B2A2B3B2BC901B801C23000
:100DB00049F058F4C13019F00E94A608CFC00E9433
:100DC0009408CCC00E94B808C9C00E949208C6C04E
:100DD000112319F08C2F817001C08695882309F4A6
:100DE000BDC02D2F229526952770220F220F6D2F23
:100DF0006F70862F90E0A0E0B0E0022E04C0880F54
:100E0000991FAA1FBB1F0A94D2F7D4FF10C04FE04E
:100E100050E060E070E004C0440F551F661F771F6C
:100E20002A95D2F7409550956095709503C040E0A3
:100E300050E0BA01C695C695C3708A019B01082B84
:100E4000192B2A2B3B2BC901B801C23049F058F4A9
:100E5000C13019F00E946B0981C00E9459097EC0FF
:100E60000E947D097BC00E94CC0878C0CF701123FE
:100E700039F08C2F0E94F2088D2F0E9497056EC0CA
:100E80008D2F0E949E058C2F0E94130967C0D23FB0
:100E900021F128F4D03F41F0D13FC1F043C0D33F0E
:100EA00019F1D43F79F03EC0112341F0053008F02C
:100EB00051C08C2F8F710E9438094CC0063008F049
:100EC00049C0F7CF80910C0382FF18C0112339F07D
:100ED0008C2F8F710E94F2083DC01123C9F38C2F13
:100EE0008F710E94130936C0112329F08C2F8F7146
:100EF0000E94DD082FC00E94D8082CC0112349F0A1
:100F0000CF718C2F0E94F20863E08C2F0E94140E88
:100F100021C081E00E942F0E0230E0F082E00E94AA
:100F20002F0E18C0112331F0002391F28D2F0E9453
:100F3000650410C0002399F2D93349F41FEF27EE5E
:100F400033E0115020403040E1F700C000008D2F09
:100F50000E940F0588EF8C0D843020F40E94D61C6F
:100F60000E94FA03DD20C9F00E94820D80FD15C0A9
:100F7000F70112820E947C0D0E94F208C7010E94B4
:100F8000EE070E947C0DDF91CF911F910F91FF9092
:100F9000EF90DF90CF900C941309DF91CF911F91C8
:100FA0000F91FF90EF90DF90CF9008950F931F93D4
:100FB000CF93DF93EC01688179818A810E94340AA2
:100FC0008C010E948F090E948008B801CE010E9406
:100FD000A505DF91CF911F910F910895CF93DF93D6
:100FE000EC01988189812B813C81232B31F08F3F4B
:100FF00031F481E09F3F19F403C081E001C080E03B
:1010000080FD1DC0CE010E949603811110C00E9478
:10101000860D8823A1F08A81882389F080910C03B2
:1010200082FD0DC082E0DF91CF910C942F0ECE0196
:101030000E94D607CE01DF91CF910C947703DF9108
:10104000CF91089580E090E00E940A1D80E090E03A
:101050000E94201D0E94AD0D0E94CF0D0E94AD1672
:101060000C947C1580910201909103010E94E21D75
:101070000C9422080E949D0D0C94320892959F704A
:10108000963079F010F4925001C09A50923068F482
:10109000803F69F018F4883E40F409C0843F29F489
:1010A00006C0883E20F0813F11F080E0089581E085
:1010B0000895FC01808191810E94290A0E943E08C6
:1010C0000895CF93DF9300D000D01F92CDB7DEB745
:1010D0000F900F900F900F900F90DF91CF91089588
:1010E000CF93DF9300D000D000D0CDB7DEB72696E7
:1010F0000FB6F894DEBF0FBECDBFDF91CF9108953C
:10110000089508950C9481080C9482080E94840824
:101110006093FB017093FC018093FD019093FE01AD
:101120000C9422080C9486080F931F930091FB01E6
:101130001091FC012091FD013091FE01602B712B7B
:10114000822B932B1F910F910C9486080F931F9362
:101150000091FB011091FC012091FD013091FE01F5
:1011600060237123822393231F910F910C9486088F
:101170000F931F930091FB011091FC012091FD0141
:101180003091FE0160277127822793271F910F91CD
:101190000C9486080C9481080E94CA086093F70199
:1011A0007093F8018093F9019093FA010C9422084E
:1011B00060E070E0CB010C94CC080F931F9341E0EA
:1011C00050E060E070E08A019B0104C0000F111F35
:1011D000221F331F8A95D2F7C901B8011F910F91C1
:1011E0000C94CC080F931F9341E050E060E070E056
:1011F00004C0440F551F661F771F8A95D2F7809150
:10120000F7019091F801A091F901B091FA018A01DA
:101210009B01082B192B2A2B3B2BC901B8011F91CD
:101220000F910C94CC080F931F9341E050E060E0C5
:1012300070E004C0440F551F661F771F8A95D2F7D0
:1012400040955095609570958091F7019091F801C7
:10125000A091F901B091FA018A019B010823192399
:101260002A233B23C901B8011F910F910C94CC088C
:101270000F931F9341E050E060E070E004C0440F22
:10128000551F661F771F8A95D2F78091F7019091BD
:10129000F801A091F901B091FA018A019B01082798
:1012A00019272A273B27C901B8011F910F910C94D8
:1012B000CC080F931F930091F7011091F801209132
:1012C000F9013091FA01602B712B822B932B1F9126
:1012D0000F910C94CC080F931F930091F70110917C
:1012E000F8012091F9013091FA01602371238223E2
:1012F00093231F910F910C94CC080F931F9300918F
:10130000F7011091F8012091F9013091FA0160275D
:101310007127822793271F910F910C94CC08089571
:1013200021E1929F800D1124E82FE695E695E69540
:10133000877051E001C0550F8A95EAF785E0E89F74
:10134000F0011124EA54FE4F20E030E070E04081CB
:10135000CB01022E02C0969587950A94E2F7817020
:10136000819584278523842781932F5F3F4F2530E4
:10137000310569F7089521E1929F800D1124682FAE
:10138000669566956695982F977085E0689FB00181
:10139000112440E050E080E0FB01E40FF51FEA5427
:1013A000FE4F208130E0092E02C0369527950A9421
:1013B000E2F721703327042E01C0220F0A94EAF7C6
:1013C000822B4F5F5F4F4530510531F70895BF9233
:1013D000CF92DF92EF92FF920F931F93CF93DF9301
:1013E0008C01C090F701D090F801E090F901F090E5
:1013F000FA018091FB019091FC01A091FD01B09157
:10140000FE01C82AD92AEA2AFB2ACFE1D0E0D70177
:10141000C6010C2E04C0B695A795979587950A949A
:10142000D2F780FD04C0219790F7B12C07C0BC2EE5
:10143000B8018C2F0E9482110197A9F38B2DDF91A7
:10144000CF911F910F91FF90EF90DF90CF90BF90C1
:101450000895CF93DF93EC010E94E709BE010E943B
:101460008211DF91CF9108951F93CF93DF93EB010A
:101470009091B501992321F0CB010E94290A13C054
:10148000882349F0CB010E94E709182F682FCE016D
:101490000E94900904C0CB010E94BB09182FBE0115
:1014A000812F0E948211DF91CF911F9108951F9388
:1014B000CF93DF93C091FF0116E080910002C8171F
:1014C00099F0D0E01C9FF0011D9FF00D1124EF5FFB
:1014D000FD4F4081518162817381848195810E9499
:1014E00070082196C770E9CFDF91CF911F910895C1
:1014F0004091310250913202609133027091340276
:1015000080913502909136020C947008EF92FF9210
:101510000F931F93CF93DF938091360282958F7044
:1015200009F065C080913302882309F460C080917E
:10153000FF01F0900002109131020091320260919F
:1015400034027091350291E01F3F09F090E0C091A4
:101550000001D0910101292F96E0E92E8F1509F4A1
:1015600046C06115710521F00F3F21F030E003C046
:1015700031E001C0322F90E030FD36C0E89EF0012E
:10158000E99EF00D1124DF01AF5FBD4F11963C9134
:101590001197301329C03C91311326C012963C910B
:1015A0001297311121C013964D915C911497461BEF
:1015B000570B4C175D07C0F4809136028F70806125
:1015C00080933602EA5FFD4F80818F708061808357
:1015D00081E392E00E94EE07DF91CF911F910F917E
:1015E000FF90EF900C94570A01968770B7CFDF9168
:1015F000CF911F910F91FF90EF9008959F92AF921E
:10160000BF92CF92DF92EF92FF920F931F93CF93EF
:10161000DF93CDB7DEB761970FB6F894DEBF0FBE8C
:10162000CDBF8C0185E0F801DE011D9601900D9281
:101630008A95E1F7D8011296EC9090913102E091F1
:10164000320220913402309135022115310531F0FA
:10165000EF3F31F481E09F3F19F403C081E001C006
:1016600080E0B82FB1709B2E80FD47C1D8014C910E
:1016700011965C9111971396AD90BC90149781E3ED
:10168000C82E82E0D82EF0903302B501621B730B96
:101690002091000130910101FF2009F4D9C080910F
:1016A00036026217730708F095C0282F207F09F0D3
:1016B00052C05E1313C0491311C0FE2CE1100EC0BE
:1016C0008F708061809336020E94780AC6010E9462
:1016D000EE0780913602F80185834DC1AB2831F0C9
:1016E0005F3F31F481E04F3F19F403C081E001C056
:1016F00080E080FD03C081E08E2502C080E090E0A4
:10170000F82FF170FF2E80FF1CC08091FF01209107
:10171000000236E0821709F40BC190E0389FF00117
:10172000399FF00D1124EF5FFD4F6181561306C004
:101730006081461303C06281E61203C00196877080
:10174000E9CFFE2CEE2009F416C1809136028160AB
:101750008093360254C05E1306C0491304C0E110E2
:1017600002C0F80199C0C8010E945908882361F19C
:10177000EE2051F120913602822F82958F7090E0F9
:10178000029774F0809131029091320298878F8392
:101790001986BB86AA862C87CE0107960E94EE0783
:1017A00086E0F801A1E3B2E001900D928A95E1F79D
:1017B0000E94860A0E94780A0AC05E1711F1C801C9
:1017C0000E94590881112CC0C8010E94EE07FF2415
:1017D000F394D1C0282F207F81F77A2DB98AA88A67
:1017E0006E2D89890E94610881E392E00E94EE07D4
:1017F00086E0D6011D928A95E9F70E94780AF12CBD
:10180000BAC04913DCCFE110DACFF8018583C801F3
:101810000E94EE0786E0D6011D928A95E9F7ABC0DB
:10182000EE2091F220913602822F82958F7090E007
:1018300002970CF4B5CF80913102909132029A83D5
:1018400089831B82BD82AC822E83CE010196A6CFF6
:101850006217730708F044C0FE2CEE2009F4B4CFE1
:101860005E1330C049132EC02091360220FD21C0E6
:10187000822F82958F70482F50E041155105C9F095
:10188000F80125834F30510541F08F5F982F9295D5
:10189000907F822F8F70892B8583C8010E94EE076D
:1018A00086E0F801A1E3B2E001900D928A95E1F79C
:1018B0003CC086E0F801A1E3B2E001900D928A9568
:1018C000E1F759C0C8010E945908811169CF809180
:1018D0003602816080933602C8010E94EE074BC039
:1018E0007A2DB98AA88A6E2D89890E94610886E0BE
:1018F000D6011D928A95E9F718C0EE2009F464CF4D
:10190000C8010E945908F82E882309F45DCF86E0AB
:10191000F801A1E3B2E001900D928A95E1F781E32D
:1019200092E00E945F040E94860A0E94780A23C007
:101930004D875E878D859E850E94290A292F2295D5
:101940002F70223028F49F7039F0811105C00BC030
:10195000243028F49F7049F4805E883020F0C8015C
:101960000E94EE079F2CF92C06C0D80115969C9179
:10197000907F91F7F8CF8F2D61960FB6F894DEBF68
:101980000FBECDBFDF91CF911F910F91FF90EF90D0
:10199000DF90CF90BF90AF909F9008951F93CF930B
:1019A000DF93CDB7DEB72C970FB6F894DEBF0FBE2E
:1019B000CDBF4F83588769877A878B879C87CE01F5
:1019C00007960E94FE0A8823D1F09F8188852A8588
:1019D0003B85232B31F08F3F31F481E09F3F19F499
:1019E00003C081E001C080E080FD47C04F81588581
:1019F00069857A858B859C850E9470083EC086E04B
:101A0000FE013796DE01119601900D928A95E1F75D
:101A1000FF81E8856A857B856115710531F0EF3FAF
:101A200031F481E0FF3F19F403C081E001C080E0A0
:101A300080FD23C02091000230E0C901019687702B
:101A400099274091FF0150E084179507F1F1F98340
:101A5000EA837D836C8396E0929FD001939FB00DC3
:101A60001124AF5FBD4FFE01319601900D929A9502
:101A7000E1F7809300020E94570A16E08091FF016F
:101A800090910002891771F1189FC00111248F5F96
:101A90009D4F0E94FE0A882329F1E091FF011E9FBD
:101AA000F0011124EF5FFD4F40815181628173810C
:101AB000848195810E9470088091FF0190E00196D9
:101AC000877099278093FF01D9CF0E943A0810921E
:101AD00000021092FF01E1E3F2E086E0DF011D92D7
:101AE0008A95E9F72C960FB6F894DEBF0FBECDBFEE
:101AF000DF91CF911F91089580915702859585952B
:101B000085950895809157028770089590915702A6
:101B1000977081E009F480E0089580917A02089539
:101B200090917A02892B80937A0208958095909102
:101B30007A02892380937A02089510927A02089596
:101B400090917902892B80937902089580959091E4
:101B50007902892380937902089510927902089579
:101B600080915802089508950C94B30D0C94B40D0F
:101B700090910C0392FD08C090915802981721F0A3
:101B8000809358020C94B60D0895809158028823D2
:101B900029F01092580280E00C94B60D0895CF936E
:101BA000DF93E0910201F091030180917A0280833A
:101BB000E0910201F0910301908180917902892BDB
:101BC000808380915802882381F0E0910201F09196
:101BD00003019081892B8083809102019091030100
:101BE0000E94361D81110E94C50DC0910201D09145
:101BF000030140E250E067E372E0CE010E94282634
:101C0000892B69F080E2FE01A7E3B2E001900D921A
:101C10008A95E1F7CE01DF91CF910C94E21CDF9120
:101C2000CF9108950C94B30D90910C0392FD10C0C8
:101C300098E0899F90011124262B209357020E943F
:101C4000F208809157028595859585950C94120E22
:101C50000C94F2081092570280E00C94120E20911E
:101C600057028095822380935702982F977099F49A
:101C700030E0482F082E000C550B2417350759F07B
:101C800090910C0392FD07C08595859585950E94DE
:101C900013090C942A0E089590910C0392FB2227AD
:101CA00020F9281769F080FB92F990930C0380913A
:101CB0000B0390910C030E949A0E82E00C942F0E5D
:101CC000089580910C0382FB882780F991E0892791
:101CD0000C944C0E81E00C944C0E80E00C944C0E55
:101CE0006FEF7FEF80E090E00C94612680E090E061
:101CF0000E943D2621E0893E9E4F09F020E0822F80
:101D0000089582E090E00C94352683E090E00C94F6
:101D10003526CF9384E090E00E943526C82F82E2DA
:101D200090E00E9435262C2F30E0A901582BCA01E3
:101D3000CF910895CF93C92F682F84E090E00E943F
:101D400043266C2F82E290E0CF910C944326AB01A6
:101D5000BC018FE090E00C945526AB01BC0183E1FF
:101D600090E00C94552660E070E0CB010C94AD0E31
:101D700060E070E0CB010E94A70E0C94B30E69EEF8
:101D80007EEF80E090E00E94612660E082E090E0DB
:101D90000E94432660E083E090E00E944326109278
:101DA000FB011092FC011092FD011092FE0160E017
:101DB00084E090E00E94432660E082E290E00E948E
:101DC000432660E085E090E00E94432660E086E0E4
:101DD00090E00E9443266FEF87E090E00E94432648
:101DE00040E050E0BA0188E090E00E94552660E0B3
:101DF0008DE090E00E94432640E050E0BA0188E187
:101E000090E00E94552660E087E190E00E94432622
:101E100040E050E0BA018CE190E00E94552660E07D
:101E200070E080E290E00E94612640E050E0BA015C
:101E300088E190E00E9455260C94B80E0C94BF0ED9
:101E4000682F8EE090E00C9443260E949E1E6093C3
:101E50009B0270939C0280939D0290939E026093DC
:101E60009702709398028093990290939A02089532
:101E70000E949E1E60939B0270939C0280939D0221
:101E800090939E02609393027093940280939502C4
:101E900090939602089585B7806885BF85B780685E
:101EA00085BF089581E008950C94520F08950C9415
:101EB000560F0C94560F0C94590F0C94560F0C940B
:101EC0005D0F0C94560F0E944B0F8EE592E10E941D
:101ED000CC1C0E94610F0C945F0F0E94570F0C9452
:101EE000560F0E9478120C94F9030E94891E0E94DA
:101EF0007C130E94710F80E00E94FC160E94691AF8
:101F00000C945B0F2F923F924F925F926F927F9251
:101F10008F929F92AF92BF92CF92DF92EF92FF92F9
:101F20000F931F93CF93DF93CDB7DEB72D970FB6E7
:101F3000F894DEBF0FBECDBF0E949113282E8111F1
:101F40000E94250F8BE792E09D878C8700E010E0D0
:101F5000302E802F0E949C122B013C01EC85FD85C8
:101F600081919191A191B191FD87EC87530142013B
:101F700088269926AA26BB2681149104A104B104BF
:101F8000B1F40F5F1F4F0630110511F78FEF8983F2
:101F90008A831B820E94921E8160782F9D838C838E
:101FA00049815A816B818D810E94150451C08091B5
:101FB0009F0281FD0E94A8121B86C12CD12C7601A4
:101FC000C394D501C4018C219D21AE21BF21892B51
:101FD0008A2B8B2B91F10E94540F8823D1F0FB8523
:101FE000FE833F824C205D206E207F2081E04528CB
:101FF0004628472809F480E088870E94921E816065
:10200000782F9A8789874E815F8168858A850E94AB
:102010001504000F111F000F111FF801E558FD4FA7
:1020200080819181A281B381C826D926EA26FB2628
:10203000C082D182E282F3820BC08B858F5F8B8757
:10204000CC0CDD1CEE1CFF1C813109F0BACF99CFFE
:1020500081E0211001C080E02D960FB6F894DEBF1C
:102060000FBECDBFDF91CF911F910F91FF90EF90E9
:10207000DF90CF90BF90AF909F908F907F906F90A8
:102080005F904F903F902F900895CF93DF930E94E1
:10209000820FD82F0E947B1AC82F81110E94380FFF
:1020A0000E94EA18D11101C0C1110E94AA170E9412
:1020B0009A15DF91CF910C940A04CF93DF930E947D
:1020C0008711EC01811521E5920708F045C08115C3
:1020D00030E5930708F094C0883E910528F5803ECE
:1020E000910508F0F8C0883A910570F4853A910599
:1020F00008F07CC08130910509F475C008F4E8C08F
:10210000049708F0E8C0E4C08F3B910508F0E0C0F8
:10211000C85AD0E0CC0FDD1FCF5ADE4F0990D881CE
:10212000C02DCE019464D8C0811540E2940758F4C4
:10213000811551E0950708F0CEC08D3E910508F459
:10214000C7C09065C9C0C11580E4D80708F4C0C0F5
:10215000DF70CE01906AC0C0811525E59207A8F412
:10216000811534E5930708F095C0811543E5940780
:1021700008F07BC0811552E5950708F061C0D82FA3
:10218000CC27CE01816F906AA7C0C11589E5D80719
:10219000A0F4C11528E5D20708F082C0C11536E5C4
:1021A000D30708F095C08C2F0E941B128F7190E00E
:1021B000D82FCC27CE0190628FC0C1154AE5D40735
:1021C00008F474C0CE0190568115904208F080C08A
:1021D0008D2F8F710E941B12DD27D0628F71AE018F
:1021E000582BCA0179C081E090E076C0C55AD0E092
:1021F000C158DE4F8881C82FD0E0CE0190646CC0FA
:1022000074E0969587957A95E1F7282F23703C2FF7
:10221000337081E090E002C0880F991F3A95E2F791
:102220009C68AC01522B9A019C2F9F7096959695B5
:1022300050E2959FE0011124C9018C2B9D2B4CC0CD
:102240008370992721E030E002C0220F331F8A9566
:10225000E2F79C2F9695969580E2989FE0011124D5
:10226000C22BD32BCE019C6837C08370992721E005
:1022700030E002C0220F331F8A95E2F79C2F96951B
:10228000969540E2949FE0011124C22BD32BCE01FE
:102290009A6822C0D82FCC27CE01846F906A1CC0C8
:1022A000DC2FCC27CE01806F906A16C08C2F8F70E8
:1022B0000E941B1294E0D695C7959A95E1F7CF70CE
:1022C000D0E0DC2FCC27D0699E01282BC90104C0A7
:1022D00080E090E001C0CE01DF91CF91089526E625
:1022E000829FC0011124FC0121E1729FE00DF11DCC
:1022F0001124E60FF11DEE0FFF1FEC53FD4F8591EA
:10230000949108950E946F110E945D100895823883
:10231000910569F1B0F48133910509F46DC048F479
:102320008932910509F463C08A32910509F469C0C4
:1023300008958533910509F455C089339105B9F0A5
:102340000895833E910569F138F4803E9105B1F01E
:10235000823E910509F10895863E9105A9F1873ED7
:102360009105B9F1843E910509F064C023C0209124
:102370000B0320FD4FC021FD4DC0089580910B033C
:1023800080FD44C080910C0380FF44C080910B030A
:1023900084FD42C083EE4DC080910B0382FF38C0A4
:1023A000F5CF80910B0382FD33C080910C0380FD3B
:1023B00031C0ECCF80910C0381FF32C080910B03C0
:1023C00084FD2AC087EE35C080910B0383FF26C0B1
:1023D000F5CF80910B0383FD21C080910C0381FD1B
:1023E0001FC0ECCF80910B0385FD1CC01DC08091E8
:1023F0000B0385FD19C016C080910B0386FD16C026
:1024000017C080910B0386FD13C010C089E311C073
:1024100082EE0FC080EE0DC080E00BC086EE09C0DA
:1024200084EE07C089E205C085E303C08AE201C0EB
:1024300081E390E0089590910B0392FF0DC0282F47
:102440002871283019F4877F846006C0282F2471F2
:10245000243011F48B7F886093FF0DC0282F2871E2
:10246000283119F4877E846106C0282F2471243115
:1024700011F48B7E886120910C0320FF0DC0382F52
:102480003871383019F4877F816006C0382F317178
:10249000313011F48E7F886021FF0DC0282F287104
:1024A000283119F4877E816106C0282F21712131DE
:1024B00011F48E7E886194FD877E089580E00895F2
:1024C0000C94700E0E9491138FE39CE90197F1F731
:1024D00000C000000E94911380E00E949C1260FFE7
:1024E00004C00E9460120C94DF1E08950C946212C6
:1024F0000E94760E811102C00E941E0F0E94810E62
:1025000080939F020E94890E90930C0380930B038B
:102510000E9476120E94850E682F70E080E090E0A5
:102520000E9492086091F7017091F8018091F90181
:102530009091FA010C94CA0824E0829FC0011124F2
:10254000FC01EB5DFC4F6081718182819381089574
:10255000089580EA8A95F1F7089500C008950C94D3
:10256000A91208950C94B1120C94B2120C94B112E9
:102570000C94B612F894E82FE295EF70F0E031A1D8
:10258000282F2F7081E090E001C0880F2A95EAF78C
:10259000982F9095932391A392A1892B82A378944D
:1025A00008950F931F93CF93DF93C3E9D1E08991EF
:1025B0008F3F11F00E94BA1281E0C939D807B9F7EC
:1025C000C2E8D1E003E911E089918F3F11F00E9448
:1025D000BA120C171D07C1F7DF91CF911F910F9110
:1025E00008954F925F926F927F928F929F92AF92D7
:1025F000BF92DF92EF92FF920F931F93CF93DF93DF
:102600008C01C62FD0E0CE018D569E4F7C01FC017F
:1026100090819F3F09F460C0D62EF894E92FE2958F
:10262000EF70F0E081A19F7021E030E001C0220F47
:102630009A95EAF7822B81A382A12095282322A3D1
:1026400078940E94AD12E2E8F1E023E931E0412CF8
:10265000512C32014394812C912C540181918F3F54
:1026600099F0A82FA295AF70B0E090964C9150E0F1
:102670008F70BA0102C0759567958A95E2F760FD83
:1026800003C0D301C20103C080E090E0DC01882ACE
:10269000992AAA2ABB2A440C551C661C771C2E17A3
:1026A0003F07E1F6F70180818F3F11F00E94BA12D7
:1026B00061E081149104A104B10409F460E08D2D5E
:1026C0000E94AF12CC0FDD1FCC0FDD1FC00FD11F3A
:1026D00088829982AA82BB82DF91CF911F910F914C
:1026E000FF90EF90DF90BF90AF909F908F907F9082
:1026F0006F905F904F9008950E94D11288E1E5E2BB
:10270000F3E0DF01982F1D929A95E9F7EDE0F3E0F1
:10271000DF011D928A95E9F786E00E94DC130C9494
:102720008203FF920F931F93CF93DF93CDB7DEB752
:1027300068970FB6F894DEBF0FBECDBF8E010F5F56
:102740001F4F88E1F80111928A95E9F7F12C6F2D5E
:10275000C8010E94F112F394F6E0FF12F8CF48E1AD
:1027600050E0B8018DE093E00E942826FF24F39406
:10277000009709F4F12C892B41F088E1F801ADE0D4
:10278000B3E001900D928A95E1F72F2D46E065E2C6
:1027900073E08DE093E00E94DD130E9484038F2D8F
:1027A00068960FB6F894DEBF0FBECDBFDF91CF9114
:1027B0001F910F91FF9008950895FF920F931F931B
:1027C000CF93DF93F82ED92F8B01C42F222349F00A
:1027D00081E08093A2020E94921E9093A1028093B6
:1027E000A0028091A2028823F1F08091A002909132
:1027F000A1020E94AA1E0597B0F0EF2DFD2FD8016F
:1028000080E090E04C2F50E08417950754F401913C
:102810001191219131910D931D932D933D9301962B
:10282000F3CF1092A202DF91CF911F910F91FF90F1
:1028300008950E94B6200E94750F0C94C2200E9439
:10284000C6200E9445100C94E0200E94301E0E9479
:102850009D200E94630F0E9419140E941F140E9461
:102860006D0FFBCF8091A90280FF06C06091090126
:1028700070E0660F771F26C081FF04C060910901D8
:1028800084E005C082FF07C06091090188E0689F6D
:10289000B001112417C09091A8029923D1F0609142
:1028A0000801961788F72091090188E0289F900178
:1028B0001124929FA001939F500D112470E0CA0132
:1028C0000E940B266038710540F46115710519F4FA
:1028D00006C068E070E0862F08958FE7089581E0D4
:1028E00008958091A90280FF08C06091050170E001
:1028F000759567957595679521C081FF06C06091B4
:10290000050170E07595679519C082FF04C060915C
:10291000050170E010C09091A702992399F0609191
:1029200004019617A0F780910501899FC001112429
:1029300070E00E940B266038710540F46115710546
:1029400019F406C061E070E0862F08958FE70895BE
:1029500081E008958D3E21F40E943214819504C0D7
:102960008E3E29F40E9432148093AD0208958F3E6A
:1029700021F40E943214819504C0803F29F40E9402
:1029800032148093AC020895893F19F40E947114A7
:1029900005C08A3F31F40E94711481958093AE0284
:1029A00008958B3F21F40E947114819504C08C3FDF
:1029B00029F40E9471148093AF0208959FE0980F4C
:1029C000983078F421E030E0A90102C0440F551F8F
:1029D0009A95E2F7CA019091AB02892B8093AB02E2
:1029E00008958D3F21F48091A90281600BC08E3F34
:1029F00021F48091A902826005C08F3F29F4809163
:102A0000A90284608093A90208958D3E39F49091C3
:102A1000AD0297FF35C01092AD0259C08E3E29F429
:102A20009091AD021916BCF32BC09091AC028F3E71
:102A300029F497FF25C01092AC0249C0803F19F4D9
:102A40001916CCF31DC09091AE02893F29F41916D6
:102A5000BCF41092AE023BC08A3F19F497FF10C03D
:102A6000F8CF8B3F39F49091AF0297FF09C01092D5
:102A7000AF022DC08C3F21F49091AF021916BCF328
:102A80009FE0980F983080F421E030E0A90102C067
:102A9000440F551F9A95E2F7CA0180959091AB02B9
:102AA00089238093AB0213C08D3F21F48091A9024A
:102AB0008E7F0BC08E3F21F48091A9028D7F05C0CF
:102AC0008F3F29F48091A9028B7F8093A902809186
:102AD000AC02811106C08091AD02811102C010923A
:102AE000A8028091AE02811106C08091AF028111CF
:102AF00002C01092A70208950E94921E2091AC027B
:102B0000211104C02091AD02222321F09093A6024E
:102B10008093A5022091AE02211104C02091AF0242
:102B2000222321F09093A4028093A3028AEA92E0E8
:102B30000C94FC1CEF92FF920F931F93CF93DF93A3
:102B400000D000D000D0CDB7DEB786E0EAEAF2E0F0
:102B5000DE01119601900D928A95E1F7E090AC02AA
:102B6000F090AD020091AE021091AF021092AC0253
:102B70001092AD021092AE021092AF02E11003C0AB
:102B8000FF2009F45DC08091A5029091A6020E94E9
:102B9000AA1EAC019091A802992339F020910A0154
:102BA00030E02417350758F04BC020910B018AE024
:102BB000289F900111242417350718F041C09F3F2A
:102BC00019F09F5F9093A802EE2061F00E943214EA
:102BD0001E1414F09FEF01C091E0989F902D1124D6
:102BE0009093AC02FF2061F00E9432141F1414F085
:102BF0009FEF01C091E0989F902D11249093AD021A
:102C00003091AC023323E1F02091AD022223C1F0D8
:102C100045EB3403C0011124992319F09093AC02C1
:102C200003C081E08093AC0235EB2303C001112483
:102C3000992319F09093AD0203C081E08093AD0217
:102C4000011103C0112309F45DC08091A30290918A
:102C5000A4020E94AA1EAC019091A702992339F008
:102C60002091060130E02417350758F04BC0209121
:102C700007018AE0289F900111242417350718F0D6
:102C800041C09F3F19F09F5F9093A702002361F01E
:102C90000E947114101614F09FEF01C091E0989FEC
:102CA000902D11249093AE02112361F00E947114B3
:102CB000111614F09FEF01C091E0989F902D112400
:102CC0009093AF023091AE023323E1F02091AF0236
:102CD0002223C1F045EB3403C0011124992319F0DC
:102CE0009093AE0203C081E08093AE0235EB2303E4
:102CF000C0011124992319F09093AF0203C081E021
:102D00008093AF028091AC0281110BC08091AD0223
:102D1000811107C08091AE02811103C08091AF0282
:102D200081110E947C15EB82FC820D831E8386E05C
:102D3000FE013196AAEAB2E001900D928A95E1F780
:102D400026960FB6F894DEBF0FBECDBFDF91CF91B0
:102D50001F910F91FF90EF900895EAEAF2E086E06C
:102D6000DF011D928A95E9F71092A8021092A7023E
:102D70001092A9020895EF92FF920F931F93CF93A1
:102D8000DF93EC017B0164E670E088E70E94C31BDF
:102D90008C01EC0EFD1ECE15DF0561F017FD0AC09B
:102DA000FE01849164E670E00E94441C8C0121962F
:102DB000892B89F30E94C81CC801DF91CF911F9114
:102DC0000F91FF90EF90089508950C94E416EDE3B1
:102DD000F3E080E092E0DF019C011D922150304041
:102DE000E1F7F0934205E09341058FEF9FEF909359
:102DF000D6028093D50208950E94E5160E94E4163B
:102E00008093D10280FD02C080E801C080E28093FF
:102E1000D0020E94BD1B6DE070E083E794E00E9449
:102E2000BB16892B11F080E008958091D10263E0F8
:102E300070E081FD03C080E794E002C08DE694E07D
:102E40000E94BB16892B79F76DE070E080E694E074
:102E50000E94BB16892B39F70E949E1EDC01CB0114
:102E6000805A9541AF4FBF4F80933D0590933E05EB
:102E7000A0933F05B09340050E94E71681E0809340
:102E8000D4028093D3021092D20208952091D002EE
:102E900036E0839FC0011124629F800D911D112493
:102EA000811522E0920714F080E090E0835C9C4F53
:102EB00090934205809341050895EF92FF920F93FE
:102EC0001F93CF93DF9320914105309142052D53FD
:102ED0003340A901460F571F4130524020F060E0B7
:102EE00072E0621B730BC091D502D091D602D9015A
:102EF000A35CBC4FA901620F731F01E010E04617ED
:102F00005707E8F4FA01E21BF30BE80FF91FE4910D
:102F1000FC91EF1781F0EC93FA01689414F8F695A0
:102F2000E7951694E1F7780102C0EE0CFF1CEA95D4
:102F3000E2F7CE29DF294F5F5F4F1196E0CFD093A4
:102F4000D602C093D502DF91CF911F910F91FF90D0
:102F5000EF9008958091D4028823F9F00E949E1E7C
:102F6000DC01CB01805A9541AF4FBF4F80933D05A7
:102F700090933E05A0933F05B09340058091D30206
:102F800081110BC062E070E08EE594E00E94BB16F8
:102F9000892B19F481E08093D3028091D3020895A4
:102FA0006F927F928F929F92AF92BF92CF92DF9259
:102FB000EF92FF920F931F93CF93DF938091D402F0
:102FC000882309F4DCC02091D5023091D602211566
:102FD000310509F4D4C08091D2028111D0C061E0E2
:102FE00070E0082F10E03B01082E02C0660C771C31
:102FF0000A94E2F7A90146215721452B11F48F5F6E
:10300000F0CF9091D102980165E0220F331F6A95AD
:10301000E1F790FD12C08295880F807680930E01B3
:10302000220F232F221F330B319520931101815E34
:1030300080930F011092120112C045E0369527953A
:103040004A95E1F7220F220F220F20930E011092D2
:103050001101295F20930F0183E08093120124E680
:1030600030E047E050E06CE071E088E70E94741CBB
:10307000892B09F084C08091D10280FD23C0A80172
:1030800095E0440F551F9A95E1F7435C5C4F04E6C9
:1030900010E020E230E060E488E70E949B1C892B6E
:1030A00009F06DC00E94AA17E301C095D0958091E8
:1030B000D5029091D602C823D923D093D602C093CB
:1030C000D5025DC080E2E0EBF2E0DF011D928A955F
:1030D000E9F785E0000F111F8A95E1F7ADE9B1E04E
:1030E00049E951E0992493942D91EA018991AE0127
:1030F000B801680F711D635C7C4F30E020553D4F77
:10310000F90197E07F01E21AF30AA92C01C0AA0C89
:10311000EA94EAF77B01B12CE70189917E018A21CB
:10312000892E8B18D82DD770CD2E0D2E000CDD08D2
:10313000C82F01C0CC0FDA95EAF7D194C194D10819
:10314000D7E0CD22DD2401C08695CA94EAF78C2B06
:10315000D0808D298083B39488E0B812DDCF915060
:1031600031969F3F79F6C1E0A13ABC0709F0BCCF88
:1031700004E610E020E230E040EB52E08CCFDF913B
:10318000CF911F910F91FF90EF90DF90CF90BF9064
:10319000AF909F908F907F906F9008958091D40210
:1031A0009091D302882389F0992369F062E070E05E
:1031B0008CE594E00E94BB16892B19F08091D30214
:1031C00008951092D3029091D30281E08927089547
:1031D0000C9428030F931F938091D402882329F124
:1031E00060E080E00E9446170E94E8180E94D01715
:1031F0008091D3028823C9F00E949E1E00913D0554
:1032000010913E0520913F0530914005DC01CB0136
:10321000801B910BA20BB30B8F3F9F4FAF4FBF474C
:1032200020F41F910F910C94CE181F910F910895C7
:10323000CF93DF93EC01FB018281882309F43CC129
:10324000C430FDE5DF0760F4CB3F9CE5D90788F487
:103250009E0122503C452431310508F02EC109C0A1
:10326000C236EDE5DE0729F0C63AFDE5DF0709F0D5
:1032700024C10E94890E90930C0380930B03C131EB
:103280008CE5D80709F4C6C008F042C0C930ECE5A7
:10329000DE0709F49BC000F5C5308CE5D80709F4BA
:1032A00085C078F4C330ECE5DE0709F478C008F097
:1032B0007AC0C230DC4509F0F5C080910B03816013
:1032C000EFC0C7309CE5D90709F478C008F07AC090
:1032D00080910B038061E4C0CD30FCE5DF0709F489
:1032E00087C058F4CB309CE5D90709F479C008F0C1
:1032F0007BC080910B0388606FC0CF30FCE5DF0797
:1033000009F480C008F082C080910B03877FC8C099
:10331000CE3F9CE5D90709F471C000F5C531FCE545
:10332000DF0709F485C068F4C3319CE5D90709F4C7
:1033300075C008F095C00E943A0880910B038F7702
:10334000AFC0CC3FFCE5DF07A9F108F054C0CB3F8C
:10335000DC4509F0A7C080910C0340C0C230EDE508
:10336000DE0709F489C058F4C1158DE5D80709F4C2
:103370005AC008F069C080910C0382602FC0C23629
:10338000EDE5DE0709F47CC0C63AFDE5DF0709F488
:1033900081C0C330DD4509F085C080E06EC08091FA
:1033A0000B0382607DC080910B0316C080910B03DC
:1033B000886076C080910C0382604FC080910B03BF
:1033C00080626EC080910B0380646AC00E943A08DC
:1033D00080910B03806864C0846062C081603DC0DE
:1033E00080910B038E7F5CC080910B038D7F58C052
:1033F00080910B0316C080910C0318C080910C03C0
:103400008D7F2BC080910B038F7E4AC080910B0370
:103410008F7D46C080910B038F7B42C080910B0350
:10342000877F8B7F3DC080910C038D7F8E7F15C081
:1034300080910B0382FB222720F991E0922790FBD9
:1034400082F990FB83F92CC080910C03982F909502
:1034500091708E7F892B90FB81F980930C0322C0A1
:103460000E943A0880910B0387FB222720F991E004
:10347000922790FB87F914C081E00E94200F12C0B0
:1034800080910B0384FB222720F991E0922790FB87
:1034900084F906C080910B03982F909590FB80F9DA
:1034A00080930B0380910B0390910C030E949A0E62
:1034B0000E943A0880E001C081E0DF91CF91089539
:1034C0008FE891E00197F1F700C0000008950C9497
:1034D0001B036898709A6998719A0E94601A8CB15F
:1034E000982F9170619902C080E001C082E0892B21
:1034F0008093D9020895E091D902EE0FEE0FE09388
:10350000D9024CB1842F817090E04CB141FB22274D
:1035100020F930E041FF02C022E030E0822B932B03
:103520008E2B8093D9028F70E82FF0E0EF55FE4F7D
:1035300090818091D802890F8093D80284305CF00A
:103540008091D7028F5F8093D70260E080E00E9475
:10355000671A21E001C020E08091D8028D3F54F429
:103560008091D70281508093D70261E080E00E9471
:10357000671A21E08091D802082E000C990B64E0B4
:1035800070E00E940B268093D802822F0895CF937B
:10359000DF9386319C4541F5EB010E948D0D982FFC
:1035A0008A812091020130910301882379F09A7A6F
:1035B00081E009F480E08093DA02911102C069E2AF
:1035C00001C065E3C9010E94CC1D0AC08091DA02E6
:1035D000811102C069E201C065E3C9010E94D71DE3
:1035E0000E94CF0D80E001C081E0DF91CF9108956E
:1035F0000F931F93CF93DF93C42FD22FFC018281AF
:103600008823C9F04093DD020E94921E9093DC0251
:103610008093DB0280E28C0F883008F057C0C770BF
:1036200081E001C0880FCA95EAF7DF91CF911F9121
:103630000F910C9497058091DD02481330C0809162
:10364000DB029091DC020E94AA1E883C910538F5AD
:1036500010E21D0FCD17B9F080E28C0F883040F4D6
:10366000C77081E001C0880FCA95EAF70E949E05E5
:10367000183028F581E09D2F977001C0880F9A952A
:10368000EAF70E949705802F0E948E051830F0F40B
:10369000D77081E001C0880FDA95EAF70AC080E2AE
:1036A0008C0F883098F4C77081E001C0880FCA95EC
:1036B000EAF7DF91CF911F910F910C949E05802F17
:1036C000DF91CF911F910F910C948E05DF91CF91D7
:1036D0001F910F9108950F939C01CB01243F4CE55E
:1036E000340731F188F4293DFCE53F07D9F02A3D44
:1036F0004CE5340779F1283D3C45A9F506E221EE79
:1037000041EE68ED7CE52BC0263FFCE53F07E1F08C
:10371000A8F0273F3C4539F507E225EE46EE67EF76
:103720007CE51DC007E225EE45EE69ED7CE517C09E
:1037300006E221EE40EE64EF7CE511C007E225EEE3
:1037400044EE65EF7CE50BC006E221EE42EE66EF4B
:103750007CE505C008E221E045EE6AED7CE50E94CB
:10376000F81A80E008C0FC018281882319F01092C9
:10377000DD0201C081E00F9108951092B9008CE044
:103780008093B80008959F92AF92BF92CF92DF923C
:10379000EF92FF920F931F93CF93DF93B82EEB011D
:1037A0000E94921E6C01C431D10558F0CF3F8FEFBB
:1037B000D80759F0CE0164E170E00E94F7257B0143
:1037C00007C0EE24E394F12C03C025E0E22EF12C97
:1037D00084E8A82E94EA992E1092BC009092BC0026
:1037E0000E94921E8C018091BC0087FD08C00E943F
:1037F000921E801B910B8E159F05A8F32AC0809105
:10380000B900887F883041F08091B900887F80318D
:1038100019F00FEF1FEF1FC0B092BB00A092BC00C9
:103820000E94921E8C018091BC0087FD08C00E94FE
:10383000921E801B910B8E159F05A8F30AC08091E4
:10384000B900887F883111F0803419F700E010E06A
:103850000EC00EEF1FEFCF3F8FEFD80709F4BCCF9C
:10386000C6010E94AA1E8C179D0708F4B5CFC80197
:10387000DF91CF911F910F91FF90EF90DF90CF904C
:10388000BF90AF909F9008950F931F93CF93DF93B6
:10389000EB018093BB0084E88093BC000E94921EE1
:1038A0008C018091BC0087FD0EC0CF3F8FEFD80701
:1038B000C1F30E94921E801B910B8C179D0788F309
:1038C0008EEF9FEF0CC02091B900287F81E090E03F
:1038D000283211F480E090E0919581959109DF9173
:1038E000CF911F910F910895CF92DF92EF92FF92A7
:1038F0000F931F93CF93DF936B018A017901B90175
:103900000E94C31BE6010C0D1D1DC017D10761F4F9
:1039100024E92093BC00DF91CF911F910F91FF907C
:10392000EF90DF90CF90089597FDF2CFB701899186
:103930000E94441CEACFCF92DF92EF92FF920F9346
:103940001F93CF93DF93C62F6A017901B8010E94BC
:10395000C31B97FD11C0B8018C2F0E94441CE601C7
:10396000EC0CFD1CCE15DF0539F097FD05C0B80144
:1039700089910E94441CF6CF24E92093BC00DF917A
:10398000CF911F910F91FF90EF90DF90CF9008950E
:1039900084E98093BC0008959093B3018093B201B1
:1039A00008959093E3028093E2020895E091E20289
:1039B000F091E302309721F00190F081E02D09941D
:1039C00080E00895E091E202F091E302309799F0EF
:1039D00020911F01222359F020910B0327FF07C0DC
:1039E000DC012C9111962C93119726E02C930280E8
:1039F000F381E02D09940895E091E202F091E30251
:103A0000309739F022E0DC012C930480F581E02D21
:103A1000099408952091E0023091E10228173907B6
:103A200071F09093E1028093E002E091E202F09164
:103A3000E302309721F00680F781E02D0994089584
:103A40002091DE023091DF022817390771F0909340
:103A5000DF028093DE02E091E202F091E302309710
:103A600021F00084F185E02D09940895FC0132963F
:103A700080911F01882331F080910B0387FF02C0E2
:103A80009EE101C096E080E0915028F02191222330
:103A9000D9F38F5FF9CF0895662351F120911F016B
:103AA0002223E9F020910B0327FF19C0462F4695EA
:103AB000469546954E31E0F4677021E030E002C053
:103AC000220F331F6A95E2F7FC01E40FF11D82819A
:103AD00090E02823392381E0232B69F409C0FC01FD
:103AE000329608962191621729F0E817F907D1F765
:103AF00080E0089581E008959C01FC0132969FEFDB
:103B000080E04191461789F09F3F19F4411101C0AF
:103B1000982F8F5F8630A9F79F3F39F0F901E90FA1
:103B2000F11D97FDFA956283089508959C012A5F1F
:103B30003F4FFC014281461301C012820196821759
:103B40009307B9F70895262F2695269526952E31A9
:103B500068F4FC01E20FF11D677021E030E001C064
:103B6000220F6A95EAF78281282B22830895262F57
:103B70002695269526952E3170F4FC01E20FF11D55
:103B8000677021E030E001C0220F6A95EAF72095C6
:103B9000828128232283089520911F01222329F066
:103BA00020910B0327FD0C94A31D0C947C1D2091E8
:103BB0001F01222329F020910B0327FD0C94B71D30
:103BC0000C94961D20911F01FC013296222331F0A6
:103BD00080910B0387FF02C08EE101C086E0DF0108
:103BE0001D928A95E9F7089508950C94F41D83E0D9
:103BF0008093E4020C94F51D811102C081E001C0A4
:103C000082E08093E4020C94F51D0C94FC1D81E08D
:103C10008093E4020C94F51D0C94071E08950C94F7
:103C20000E1E0C940F1E0C940E1E0C940E1E0C9463
:103C30000E1ECF930E94151E0E9491130E94131E08
:103C4000C0E08C2F0E949C12672B682B692B29F4F3
:103C5000CF5FC630B1F780E001C081E0CF91089519
:103C600008951F920F920FB60F9211248F939F9376
:103C7000AF93BF938091E502811113C080914305FA
:103C800090914405A0914505B09146054196A11D2E
:103C9000B11D8093430590934405A0934505B093CF
:103CA0004605BF91AF919F918F910F900FBE0F90DE
:103CB0001F90189580914B05843031F10E94E803E4
:103CC0001092E50220E488E190E00FB6F894A89500
:103CD000809360000FBE2093600083B7817F846073
:103CE00083BF83B7816083BF7894889583B78E7FC5
:103CF00083BF0FB6F894A895809160008861809387
:103D00006000109260000FBE08950E943A080C9463
:103D1000EE0382E084BD93E095BD9AEF97BD80935A
:103D20006E0008952FB7F894809143059091440553
:103D3000A0914505B09146052FBF08952FB7F8947F
:103D40006091430570914405809145059091460529
:103D50002FBF08959C014FB7F8948091430590912F
:103D60004405A0914505B09146054FBF821B930BBA
:103D7000089578941F920F920FB60F9211248F938B
:103D80009F93AF93BF938091430590914405A09179
:103D90004505B09146050196A11DB11D80934305CF
:103DA00090934405A0934505B0934605BF91AF910C
:103DB0009F918F910F900FBE0F901F901895F894C0
:103DC00081E08093E00080E28093D800E9ECF0E0AD
:103DD00010828FE19EE40197F1F700C000001DBA48
:103DE000109268001CBC10BE1FBA10927A0010928C
:103DF0006E0010926F00109270001092710010828D
:103E00001092BC0011B814B817B81AB81DB810BA7F
:103E100012B815B818B81BB81EB811BA0C9400FE29
:103E20000895809109030895089522E02093E90000
:103E30002FEF3091E800215035FD06C035ED3A9561
:103E4000F1F700002111F5CF2091E80025FF0BC00C
:103E500040E050E066E070E00E9452218091E8006E
:103E60008E778093E8000895CF93DF9320911F0110
:103E7000222339F020910B0327FF03C060E222E0E8
:103E800002C068E021E02093E9002FEF3091E800C4
:103E9000215035FD06C035ED3A95F1F700002111AE
:103EA000F5CF2091E80025FF1DC0EC0180911F0196
:103EB000811105C040E050E068E070E003C070E0B0
:103EC00040E050E0CE010E9452218091E8008E77C0
:103ED0008093E80080E2FE01A9EEB2E001900D922D
:103EE0008A95E1F7DF91CF9108958093E602709370
:103EF000E8026093E70280914B05843001F582E08F
:103F00008093E9008FEF9091E800815095FD06C005
:103F100095ED9A95F1F700008111F5CF8091E800B9
:103F200085FF0DC040E050E063E070E086EE92E077
:103F30000E9452218091E8008E778093E8000895D6
:103F4000BC0184E00C94751FBC0183E00C94751FC8
:103F500080914A05811109C00E94DF220E944123FD
:103F60008091E20084608093E200089510924A05F7
:103F700008950C940C1E6091470581E0611101C009
:103F800080E00C94F71D90914B0581E0943009F08E
:103F900080E0609147050C94FC1D42E061EC81E0FB
:103FA0000E94582242E261EC82E00E9458229091E5
:103FB0004B0581E0943009F080E0609147050C9456
:103FC000051E80914D05833009F45FC030F48130C7
:103FD00071F0823009F498C008958A3009F484C0E1
:103FE0008B3009F46AC0893009F0A6C020C08091E6
:103FF0004C05813A09F0A0C08091E800877F80934A
:10400000E8008091500590915105892B21F460E2E0
:1040100089EE92E003C060E080E090E070E00E94F2
:104020009D218091E8008B778093E800089580912E
:104030004C05813209F080C0809150059091510566
:10404000029708F079C08091E800877F8093E800AC
:104050008091E80082FD05C080914B058111F8CF69
:104060006BC08091F2009091F300029731F480913F
:10407000F100813011F0863021F48091F1008093BD
:1040800009038091E8008B7753C080914C05813AF9
:1040900009F052C08091500590915105892B09F08B
:1040A0004BC08091E800877F8093E8008091E80012
:1040B00080FFFCCF80911F0136C080914C0581327A
:1040C000D9F58091500590915105892BA9F58091E2
:1040D000E800877F8093E8000E948D2280914E0542
:1040E00080931F010C943A0880914C05813221F590
:1040F0008091E800877F8093E8000E948D22809164
:104100004F0580930A03089580914C05813AA1F4EC
:104110008091E800877F8093E8008091E80080FF2D
:10412000FCCF80910A038093F1008091E8008E77A4
:104130008093E8000C948D22089584B7877F84BF14
:104140000FB6F894A8958091600088618093600014
:10415000109260000FBE90E080E80FB6F894809354
:104160006100909361000FBE0C94071E0E94DF2235
:104170000E944123E2EEF0E08081846080837894A5
:104180000C94DC2583E191E00C94D11C80914B05CB
:104190008530A9F480914B05853079F40E945A1E30
:1041A000809149058823B1F30E94191E882391F359
:1041B0000E943C210E943A08EDCF0C94851E089580
:1041C00008950C94E320292F332723303105C9F0BB
:1041D00060F42130310581F02230310509F044C00E
:1041E0008BE390E020EB34E043C021323105E1F075
:1041F0002232310549F138C082E190E02BEE34E003
:1042000037C099278130910549F028F0029761F570
:10421000E0E8F4E005C0ECEAF4E002C0E6E9F4E02E
:10422000849190E09F0124C06115710541F06130D7
:104230007105D1F489E090E02BED34E019C089E0FC
:1042400090E022EC34E014C06115710541F061305A
:10425000710551F486EB90E02DEF34E009C080E465
:1042600090E023EB35E004C080E090E020E030E017
:10427000FA0131832083089584E189BD86E189BDF7
:1042800009B400FEFDCF8091D8008F7D8093D800C7
:104290008091E00082608093E0008091E00081FDE9
:1042A000FCCF0895CF92DF92EF92FF920F931F936E
:1042B000CF93DF93EC018B017A010E94AC22811134
:1042C00033C0E114F10439F0F70180819181081BBA
:1042D000190BC80FD91FC12CD12C0115110519F1CB
:1042E0008091E80085FD16C08091E8008E7780936C
:1042F000E800E114F10449F0F70180819181C80ED2
:10430000D91ED182C08285E00FC00E94AC228823D2
:1043100021F30AC089918093F10001501109FFEF48
:10432000CF1ADF0ADACF80E0DF91CF911F910F9192
:10433000FF90EF90DF90CF9008952091520530913B
:1043400053052617370748F06115710539F4209198
:10435000E8002E772093E80001C0B901FC0120E0BD
:104360006115710569F180914B058823E1F1853074
:10437000E1F18091E80083FD3AC08091E80082FD80
:104380002CC08091E80080FFEBCF8091F2009091EB
:10439000F3006115710551F08830910538F42191D1
:1043A0002093F100615071090196F3CF21E0089745
:1043B00009F020E08091E8008E778093E800D0CF6C
:1043C0002111D1CF0AC080914B05882361F085303F
:1043D00061F08091E80083FD0AC08091E80082FFCF
:1043E000F2CF80E0089582E0089583E0089581E0AF
:1043F000089520915205309153052617370748F04C
:104400006115710539F42091E8002E772093E800BA
:1044100001C0B901FC0120E06115710581F18091B5
:104420004B05882309F43EC0853009F43DC08091D6
:10443000E80083FD3BC08091E80082FD2DC08091A3
:10444000E80080FFE9CF8091F2009091F3006115C0
:10445000710559F08830910540F424912093F100C2
:104460003196615071090196F2CF21E0089709F069
:1044700020E08091E8008E778093E800CDCF211175
:10448000CECF0AC080914B05882361F0853061F062
:104490008091E80083FD0AC08091E80082FFF2CF9E
:1044A00080E0089582E0089583E0089581E0089512
:1044B000982F973068F59093E900981739F070912C
:1044C000EC002091ED005091F00003C0242F762FD6
:1044D00050E021FD02C09F5FECCF3091EB003E7FAA
:1044E0003093EB003091ED003D7F3093ED00309143
:1044F000EB0031603093EB007093EC002093ED0003
:104500005093F0002091EE0027FDE5CF80E0089564
:104510008F708093E90081E0089580914C0587FFBA
:1045200011C08091E80082FD05C080914B0581118A
:10453000F8CF11C08091E8008B770BC080914B05BC
:10454000882349F08091E80080FFF8CF8091E8004F
:104550008E778093E80008952091E4003091E50083
:1045600095E64091EC00842F817040FF23C080913C
:10457000E80080FD1DC080914B05882399F08530AF
:1045800099F08091EB0085FD11C04091E4005091BD
:10459000E5002417350729F3915011F09A01E1CF76
:1045A00084E0089582E0089583E0089581E008950D
:1045B00080E008954091E80042FFDDCF08950E9419
:1045C00050230E945823E0EEF0E0808181608083D8
:1045D000E8EDF0E080818F77808319BCA7EDB0E033
:1045E0008C918E7F8C9380818F7E808310924A0580
:1045F00008950F931F93CF93DF930E9450230E943F
:104600005823C8EDD0E088818F77888388818068BF
:10461000888388818F7D8883E7EDF0E080818068E2
:10462000808319BC10924B051092470510924905E2
:104630001092480500EE10E0F80180818B7F8083A6
:1046400088818160888342E060E080E00E94582297
:10465000E1EEF0E080818E7F8083E2EEF0E0808109
:1046600081608083808188608083F80180818E7F73
:104670008083888180618883DF91CF911F910F9122
:104680000895E8EDF0E080818F7E8083E7EDF0E033
:1046900080818160808381E080934A050C94F922B7
:1046A000E8EDF0E080818C7F80831092E200089535
:1046B0001092DA001092E10008951F920F920FB647
:1046C0000F9211240BB60F922F933F934F935F934A
:1046D0006F937F938F939F93AF93BF93EF93FF93CA
:1046E0008091E10082FF0BC08091E20082FF07C051
:1046F0008091E1008B7F8093E1000E94DB25809117
:10470000DA0080FF1FC08091D80080FF1BC080911D
:10471000DA008E7F8093DA008091D90080FF0DC08F
:1047200084E189BD86E189BD09B400FEFDCF81E049
:1047300080934B050E94A81F05C019BC10924B0521
:104740000E94B61F8091E10080FF19C08091E200B5
:1047500080FF15C08091E2008E7F8093E2008091FF
:10476000E20080618093E2008091D80080628093B3
:10477000D80019BC85E080934B050E94BB1F809137
:10478000E10084FF30C08091E20084FF2CC084E10E
:1047900089BD86E189BD09B400FEFDCF8091D800B6
:1047A0008F7D8093D8008091E1008F7E8093E1001F
:1047B0008091E2008F7E8093E2008091E200816030
:1047C0008093E20080914705882311F084E007C0C0
:1047D0008091E30087FD02C081E001C083E0809307
:1047E0004B050E94C31F8091E10083FF29C0809187
:1047F000E20083FF25C08091E100877F8093E10084
:1048000082E080934B05109247058091E1008E7FF6
:104810008093E1008091E2008E7F8093E20080919E
:10482000E20080618093E20042E060E080E00E946C
:1048300058228091F00088608093F0000E94B91F98
:10484000FF91EF91BF91AF919F918F917F916F9168
:104850005F914F913F912F910F900BBE0F900FBE24
:104860000F901F9018951F920F920FB60F92112460
:104870000BB60F922F933F934F935F936F937F935A
:104880008F939F93AF93BF93CF93DF93EF93FF9358
:10489000C091E900CF708091EC00D82FD17080FDDD
:1048A000D0E81092E9008091F000877F8093F000BB
:1048B00078940E947B241092E9008091F000886037
:1048C0008093F000CD2BCF70C093E900FF91EF9162
:1048D000DF91CF91BF91AF919F918F917F916F9118
:1048E0005F914F913F912F910F900BBE0F900FBE94
:1048F0000F901F9018951F93CF93DF93CDB7DEB71E
:10490000AA970FB6F894DEBF0FBECDBFECE4F5E07A
:104910008091F100819325E0E435F207C9F70E9408
:10492000E11F8091E80083FF2EC180914C0590919A
:104930004D05492F50E04A30510508F024C1FA01D5
:10494000E85AFF4F0C941F26803821F0823809F076
:104950001AC108C08091480590914905992389F0B2
:1049600082600FC0809150058F70873008F00BC1B6
:104970008093E9008091EB0085FB882780F91092F5
:10498000E9009091E800977F9093E8008093F10010
:104990001092F100D1C0282F2D7F09F0F4C0882398
:1049A00019F0823061F0EFC080914E05813009F03E
:1049B000EAC0933009F080E0809349052EC08091D1
:1049C0004E0581112AC0809150058F702FEF280F5E
:1049D000263008F0D8C08093E9002091EB0020FF3A
:1049E0001CC0933021F48091EB00806214C0909140
:1049F000EB0090619093EB0021E030E0A90102C050
:104A0000440F551F8A95E2F74093EA001092EA009E
:104A10008091EB0088608093EB001092E900809118
:104A2000E800877F8093E8000E948D22ACC081114E
:104A3000AAC010914E051F778091E3008078812BEA
:104A40008093E3008091E800877F8093E8000E94D4
:104A50008D228091E80080FFFCCF8091E300806888
:104A60008093E300111102C082E001C083E08093D3
:104A70004B0589C08058823008F085C080914E0572
:104A800090914F058C3D53E0950779F583E08A833B
:104A90008AE289834FB7F894DE01139620E03EE066
:104AA00051E2E32FF0E050935700E49120FF03C060
:104AB000E295EF703F5FEF708E2F90E0EA3010F0DC
:104AC000C79601C0C0968D939D932F5F243149F7FF
:104AD0004FBF8091E800877F8093E8006AE270E032
:104AE000CE0101960E949D2116C0609150057091E3
:104AF0005105AE014F5F5F4F0E94E120BC01892B41
:104B000009F441C09091E800977F9093E800898173
:104B10009A810E94F9218091E8008B778093E800C8
:104B200032C0803881F58091E800877F8093E8006B
:104B3000809147058093F1008091E8008E7772CFD5
:104B4000811121C080914E0590914F0599270297C0
:104B5000D4F48091E800877F8093E80080914E052F
:104B6000809347050E948D2280914705811106C0E0
:104B70008091E30087FD02C081E001C084E0809362
:104B80004B050E94CD1F8091E80083FF0AC08091F1
:104B9000E800877F8093E8008091EB00806280933B
:104BA000EB00AA960FB6F894DEBF0FBECDBFDF9123
:104BB000CF911F9108950895CF9380914B0588233D
:104BC000A1F0C091E900CF709091EC00892F817025
:104BD00090FD80E8C82B1092E9008091E80083FDE9
:104BE0000E947B24CF70C093E900CF910895AA1B47
:104BF000BB1B51E107C0AA1FBB1FA617B70710F0C8
:104C0000A61BB70B881F991F5A95A9F780959095F9
:104C1000BC01CD01089597FB072E16F4009407D030
:104C200077FD09D00E94F72507FC05D03EF490954A
:104C300081959F4F0895709561957F4F0895EE0F70
:104C4000FF1F0024001C0BBE0790F691E02D099475
:104C5000FB01DC0104C08D910190801921F44150C9
:104C60005040C8F7881B990B0895F999FECF92BD63
:104C700081BDF89A992780B50895A8E1B0E042E097
:104C800050E00C946926262FF999FECF92BD81BD84
:104C9000F89A019700B4021639F01FBA20BD0FB67A
:104CA000F894FA9AF99A0FBE08950396272F0E9456
:104CB00044260E944326252F0E944426242F0C942C
:104CC00044260196272F0E9444260C944326DC019B
:104CD000CB01FC01F999FECF06C0F2BDE1BDF89A07
:104CE000319600B40D9241505040B8F70895F894B1
:024CF000FFCFF4
:104CF200C8005902280850011E0A14010021007F31
:104D0200220003111F341F151FA41FA01F141F010F
:104D1200E200E900EA00B500B600B700CD00830169
:104D2200CC008A019201940121022302240225026D
:104D3200260227022A02B300B4006F0070008182AB
:104D420083E200E900EA00B500B600B700CD0083B7
:104D520001CC008A0192019401210223022402253E
:104D620002260227022A02B300B4006F00700081FB
:104D7200828336353433323130C7C6F0F1F2F3F480
:104D8200F5F6F76061626364650008101818100890
:104D92000000FF0100010000FFFF0000010001FF11
:024DA20000000F
:00000001FF
